:100000000C9483000C94A4000C94A4000C94A40001
:100010000C94A4000C94A4000C94A4000C94A400D0
:100020000C94A4000C94A4000C94A4000C94A400C0
:100030000C94A4000C94A4000C94A4000C94A400B0
:100040000C94A4000C94A4000C94A4000C94A400A0
:100050000C94A4000C94A4000C94A4000C94A40090
:100060000C94A4000C946C020C94BC010C94A4009D
:100070000C94A4000C94A4000C94A4000C94A40070
:100080000C94A4000C94A4000C94A4000C94A40060
:100090000C9440020C9490010C94A4000C94A400C5
:1000A0000C94A4000C94A4000C94A4000C94A40040
:1000B0000C94A4000C94A4000C94A4000C94A40030
:1000C0000C94A4000C94A4000C94A4000C941402AE
:1000D0000C9464010C94A4000C94E8010C94380175
:1000E0000C94A40045464765666700202B2D2E30F2
:1000F00031323334353637383968006364696E6FAE
:1001000070737578580011241FBECFEFD1E2DEBFA7
:10011000CDBF00E00CBF12E0A0E0B2E0E6E6F6E101
:1001200000E00BBF02C007900D92AC32B107D9F7C7
:1001300012E0ACE2B2E001C01D92A034B107E1F7D9
:100140000E94A6000C94310B0C9400000F93CF93E7
:10015000DF9380E884B985B1805885B984E690E062
:100160000E94980285B1805885B984E690E00E948B
:10017000980285B1805885B984E690E00E94980283
:1001800085B1805885B984E690E00E94980280E0AD
:1001900040E056E960E070E028E208E20E94D10207
:1001A000BC019093350280933402789480E092E011
:1001B0000E94680ACEE0D2E080913402909135022C
:1001C0000E94D604882309F44BC080913402909198
:1001D00035020E94E909082F8DB79EB708970FB620
:1001E000F8949EBF0FBE8DBFEDB7FEB731968091DC
:1001F000340290913502ADB7BEB712969C938E93A0
:100200001197D383C28304831582068317820E94C9
:100210002B0A8DB79EB708960FB6F8949EBF0FBEF7
:100220008DBF063619F00337D9F40CC000E085B154
:10023000805885B984E690E00E9498020F5F0830EC
:10024000B1F70EC085B1805885B988EE93E00E9461
:10025000980285B1805885B988EE93E00E94980293
:1002600085B1805885B98AEF90E00E949802A4CFAA
:100270001F920F920FB60F920BB60F9211242F936D
:100280003F934F935F936F937F938F939F93AF931E
:10029000BF93EF93FF9380913202909133020E94BB
:1002A0008504FF91EF91BF91AF919F918F917F91C5
:1002B0006F915F914F913F912F910F900BBE0F90D7
:1002C0000FBE0F901F9018951F920F920FB60F92AE
:1002D0000BB60F9211242F933F934F935F936F931D
:1002E0007F938F939F93AF93BF93EF93FF938091EF
:1002F0003002909131020E948504FF91EF91BF91ED
:10030000AF919F918F917F916F915F914F913F91AD
:100310002F910F900BBE0F900FBE0F901F9018954E
:100320001F920F920FB60F920BB60F9211242F93BC
:100330003F934F935F936F937F938F939F93AF936D
:10034000BF93EF93FF9380912E0290912F020E9412
:100350008504FF91EF91BF91AF919F918F917F9114
:100360006F915F914F913F912F910F900BBE0F9026
:100370000FBE0F901F9018951F920F920FB60F92FD
:100380000BB60F9211242F933F934F935F936F936C
:100390007F938F939F93AF93BF93EF93FF9380913E
:1003A0002C0290912D020E948504FF91EF91BF9144
:1003B000AF919F918F917F916F915F914F913F91FD
:1003C0002F910F900BBE0F900FBE0F901F9018959E
:1003D0001F920F920FB60F920BB60F9211242F930C
:1003E0003F934F935F936F937F938F939F93AF93BD
:1003F000BF93EF93FF9380913202909133020E945A
:100400003804FF91EF91BF91AF919F918F917F91B0
:100410006F915F914F913F912F910F900BBE0F9075
:100420000FBE0F901F9018951F920F920FB60F924C
:100430000BB60F9211242F933F934F935F936F93BB
:100440007F938F939F93AF93BF93EF93FF9380918D
:100450003002909131020E943804FF91EF91BF91D8
:10046000AF919F918F917F916F915F914F913F914C
:100470002F910F900BBE0F900FBE0F901F901895ED
:100480001F920F920FB60F920BB60F9211242F935B
:100490003F934F935F936F937F938F939F93AF930C
:1004A000BF93EF93FF9380912E0290912F020E94B1
:1004B0003804FF91EF91BF91AF919F918F917F9100
:1004C0006F915F914F913F912F910F900BBE0F90C5
:1004D0000FBE0F901F9018951F920F920FB60F929C
:1004E0000BB60F9211242F933F934F935F936F930B
:1004F0007F938F939F93AF93BF93EF93FF938091DD
:100500002C0290912D020E943804FF91EF91BF912F
:10051000AF919F918F917F916F915F914F913F919B
:100520002F910F900BBE0F900FBE0F901F9018953C
:10053000EF92FF920F931F93A0E0B0E0BC01CD01BA
:1005400020EA3FE040E050E00E941D087B018C0162
:10055000C801AA27BB27A0E0B0E020E030E040E0DF
:1005600050E060E070E007C0FB013197F1F72F5FCA
:100570003F4F4F4F5F4F281739074A075B07A0F3DC
:10058000C801B701807090706115710581059105F2
:1005900019F0CB010197F1F71F910F91FF90EF90A8
:1005A00008959F92AF92BF92CF92DF92EF92FF9207
:1005B0000F931F93CF93DF93982E6A017B01B22E86
:1005C000A02E81E0821708F0AAC0081709F4A7C07E
:1005D00089E090E00E9485088C01FC019082B18244
:1005E000A2821482848183831682868185838B2DE7
:1005F00090E08A0D911D0E948508EC01F80190871A
:10060000878384E0CC0CDD1CEE1CFF1C8A95D1F79F
:1006100060E074E284EF90E0A70196010E944F0829
:1006200021503040F1E09F1621F19F1640F082E00A
:100630009816C9F1E3E09E1609F069C04EC088E142
:100640008093C1003093C5002093C4008EE993E0ED
:100650006CE174E00E949D09FC01158704871093EA
:100660002D0200932C028091C10080688093C1000C
:1006700058C088E18093C9003093CD002093CC000E
:100680008EE993E06CE174E00E949D09FC011587FE
:10069000048710932F0200932E028091C900806876
:1006A0008093C9003EC088E18093D1003093D5008B
:1006B0002093D4008EE993E06CE174E00E949D09E0
:1006C000FC0115870487109331020093300280915A
:1006D000D10080688093D10024C088E180933101EB
:1006E00030933501209334018EE993E06CE174E09E
:1006F0000E949D09FC011587048710933302009323
:100700003202809131018068809331010AC02097C4
:1007100019F0CE010E943209C8010E943209E0E0BE
:10072000F0E0CF01DF91CF911F910F91FF90EF90FB
:10073000DF90CF90BF90AF909F9008950F931F933D
:10074000CF93DF93382FFB01C485D5856A81623052
:1007500008F446C0E62FF0E08F01015010408E8172
:100760002D81AF01480F511DCA01821B9109BF01A4
:100770000E943C088017910791F38E819981EF8147
:10078000F885E80FF11DE90FF11D30838E8190E0AF
:100790006A81019670E00E943C088E8388818130D6
:1007A00069F0813028F0823079F08330F1F512C0A1
:1007B0008091C10080628093C10037C08091C900E0
:1007C00080628093C90031C08091D10080628093A3
:1007D000D1002BC08091310180628093310125C00E
:1007E0008881813071F0813028F0823089F0833047
:1007F000E1F415C08091C00085FFFCCF3093C600A6
:1008000014C08091C80085FFFCCF3093CE000DC08E
:100810008091D00085FFFCCF3093D60006C0809138
:10082000300185FFFCCF3093360180E090E0DF910E
:10083000CF911F910F910895CF93DF93FC01C48551
:10084000D5859B818C819817E1F38B81EF81F885A9
:10085000E80FF11D20818B8190E06981019670E0A5
:100860000E943C088B83822F90E0DF91CF91089506
:100870001F93CF93DF93EC018881813071F0813039
:1008800028F0823089F08330E1F415C08091C000F7
:1008900087FF37C01091C60014C08091C80087FF41
:1008A00030C01091CE000DC08091D00087FF29C0CC
:1008B0001091D60006C08091300187FF22C01091B0
:1008C0003601298130E08C814B81B901680F711D9F
:1008D000CB01841B9109B9010E943C082150304092
:1008E0008217930774F48C81EF81F885E80FF11D6E
:1008F00010838C8190E06981019670E00E943C0831
:100900008C83DF91CF911F910895CF93DF93EC01FA
:100910009D818E812881981709F5213069F0213059
:1009200028F0223079F02330F1F512C08091C10017
:100930008F7D8093C10037C08091C9008F7D8093E7
:10094000C90031C08091D1008F7D8093D1002BC030
:10095000809131018F7D8093310125C09D818981F6
:10096000EF81F885E80FF11DE90FF11DE0818D8120
:1009700090E06A81019670E00E943C088D832130EE
:1009800051F0213028F0223049F0233061F409C0C1
:10099000E093C60008C0E093CE0005C0E093D60007
:1009A00002C0E0933601DF91CF910895DC011C96DF
:1009B000ED91FC911D979381848120E0981321E0B3
:1009C000822F08956F927F928F929F92AF92BF92E3
:1009D000CF92DF92EF92FF920F931F93DF93CF930B
:1009E000CDB7DEB72B970FB6F894DEBF0FBECDBFE5
:1009F0005C014B017A01FC0117821682838181FD23
:100A000008C06FEF7FEF08C142E050E0E40EF51E32
:100A100004C03E010894611C711CF501D380F401EF
:100A2000D3FC8591D3FE81914F01882309F4F1C055
:100A3000853259F4D3FC6591D3FE61914F01653243
:100A400019F0062F10E01BC085E290E02BC00023B8
:100A500009F4DFC08BEE90E0602F70E00E949209F5
:100A6000892B39F4033211F4106103C00C3661F4A0
:100A70001068F401D3FC0591D3FE01914F0117FFDB
:100A8000E6CF002309F4C5C084EE90E0602F70E04B
:100A90000E949209892B51F044E050E0E40EF51ECB
:100AA0008FE390E0B5010E943C0AB7CF033629F0EE
:100AB000033779F00335F1F40BC087010E5F1F4F48
:100AC000F70180819181B5010E943C0A7801A5CF90
:100AD0001160F701C080D18004C090E0B5010E9490
:100AE0003C0AF60110FD859110FF81916F0188236A
:100AF000A1F78ACF043611F0093639F517FF08C07F
:100B0000F701208131814281538184E090E00AC065
:100B1000F701808191819C01442737FD4095542F36
:100B200082E090E0E80EF91E1F7E57FF08C0509546
:100B30004095309521953F4F4F4F5F4F1064CA014C
:100B4000B901A3012AE030E034C00037A9F0013731
:100B500030F40835B1F00F3609F05BC006C0053738
:100B600039F0083709F055C008C028E030E00CC063
:100B70001F7E2AE030E008C01061146220E130E0FE
:100B800003C0146020E132E017FF08C0F701608164
:100B900071818281938144E050E008C0F701808137
:100BA0009181BC0180E090E042E050E0E40EF51E4F
:100BB000A3010E94AD0AD82ED618012F10E006FF1F
:100BC00005C08DE290E0B5010E943C0A04FF15C00B
:100BD000FE01ED0DF11D8081803379F080E390E01E
:100BE000B5010E943C0A02FF08C000721070C801E3
:100BF000885A9F4FB5010E943C0ADA94F301ED0D2B
:100C0000F11D808190E0B5010E943C0ADD20A9F72A
:100C100004CFF50166817781CB012B960FB6F8944E
:100C2000DEBF0FBECDBFCF91DF911F910F91FF901F
:100C3000EF90DF90CF90BF90AF909F908F907F907C
:100C40006F900895FC0120FD08C023FD05C022FF20
:100C500002C073836283518340830895EF92FF92B1
:100C60000F931F9344FF02C033E011C046FF02C040
:100C700034E00DC0DB01FC01AA0FBB1FEE1FFF1FFC
:100C80001094D1F76A0F7B1F8E1F9F1F31E0660FF4
:100C9000771F881F991F3150D1F77B018C01E20E1D
:100CA000F11C011D111DA8019701B701CA011F9177
:100CB0000F91FF90EF9008950F931F93CF93DF93C1
:100CC0008C01C8010E94E909EC0197FD08C00E944F
:100CD0008A09892BB1F7CE01B8010E94930ACE018F
:100CE000DF91CF911F910F910895AF92BF92CF9254
:100CF000DF92EF92FF920F931F93CF93DF93EC015C
:100D0000C62E5A01122F0E94E909AC018B3219F04C
:100D10008D3251F41068CA9409F46DC0CE010E945E
:100D2000E909AC0197FD67C06DEFD62ED1228D2D5C
:100D3000807301F54033F1F4CA9409F447C0CE0141
:100D40000E94E909AC0197FD41C082E0D82A4837EA
:100D500011F0483559F480E4D82ACA94B9F1CE018B
:100D60000E94E909AC0199232CF430C0D6FC02C0E2
:100D700080E1D82AEE24FF248701242F2053283035
:100D800088F0D4FC09C02A3068F0D6FE05C02F7D5B
:100D9000822F8151863028F0CA01BE010E94930A39
:100DA00012C02750C801B7014D2D0E942E067B01AD
:100DB0008C0182E0D82ACA9461F0CE010E94E90930
:100DC000AC0197FFDACFD1FC04C015C0EE24FF249C
:100DD0008701D7FE08C010950095F094E094E11CBF
:100DE000F11C011D111DC501B801A7012D2D0E9487
:100DF000220681E001C080E0DF91CF911F910F9129
:100E0000FF90EF90DF90CF90BF90AF9008956F92DA
:100E10007F928F929F92AF92BF92CF92DF92EF928A
:100E2000FF920F931F93CF93DF935C016B013A0105
:100E3000FC01178216828824DDC0812F90E00E9479
:100E40008A09892B21F0C5010E945C06D3C01532A6
:100E500049F4F601F3FC6591F3FE61916F0165328F
:100E600069F415E2C5010E94E90997FDCFC0181782
:100E700009F4C0C0B5010E94930ACDC06A3219F0CE
:100E8000162F00E006C0F3FC1591F3FE11916F01DF
:100E900001E099240FC00260692D70E080E090E0CD
:100EA00040E20E942E06962EF601F3FC1591F3FE09
:100EB00011916F01212F20532A3068F301FD03C0E7
:100EC00099249A9403C0992009F4A5C0183621F0FA
:100ED0001C3699F4F6010BC0F601F3FC6591F3FEA4
:100EE0006191683619F06F01162F07C00860046021
:100EF000F3FC1591F3FE11916F01112309F48BC0DE
:100F00008BEF90E0612F70E00E949209892B09F429
:100F100082C0802F00FF03C0EE24FF2407C0F3012E
:100F2000E080F18022E030E0620E731E1E3651F444
:100F3000F5014681578160E070E0C701202F0E94D3
:100F4000220658C0133691F481FD02C0992493946F
:100F5000C5010E94E90997FD59C0E114F10419F097
:100F6000F70181937F019A9499F742C0C5010E94CD
:100F70005C0697FD4BC01F3659F1103728F4143624
:100F800029F1193639F527C0133719F0153711F53E
:100F90001DC0C5010E94E909EC0197FD11C00E9426
:100FA0008A09892B29F0CE01B5010E94930A08C055
:100FB000E114F10419F0F701C1937F019A9449F704
:100FC000E114F104A9F0F701108212C0006203C01D
:100FD000006101C00064C501692DA701202F0E9496
:100FE0007506882329F4F5018381807379F413C091
:100FF00000FF8394F501F380F601F3FC1591F3FEF5
:1010000011916F01112309F018CF05C0882019F440
:101010002FEF3FEF02C0282D30E0C901DF91CF91C3
:101020001F910F91FF90EF90DF90CF90BF90AF9006
:101030009F908F907F906F900895629FD001739FD3
:10104000F001829FE00DF11D649FE00DF11D929F64
:10105000F00D839FF00D749FF00D659FF00D9927A3
:10106000729FB00DE11DF91F639FB00DE11DF91FC7
:10107000BD01CF011124089597FB092E07260AD040
:1010800077FD04D02ED006D000201AF4709561951B
:101090007F4F0895F6F7909581959F4F0895A1E2AF
:1010A0001A2EAA1BBB1BFD010DC0AA1FBB1FEE1FE2
:1010B000FF1FA217B307E407F50720F0A21BB30B2D
:1010C000E40BF50B661F771F881F991F1A9469F7A9
:1010D00060957095809590959B01AC01BD01CF0105
:1010E0000895AA1BBB1B51E107C0AA1FBB1FA6176F
:1010F000B70710F0A61BB70B881F991F5A95A9F7C1
:1011000080959095BC01CD010895CF93DF93BC01EC
:101110008230910510F462E070E0A0913802B09145
:101120003902ED01E0E0F0E040E050E021C08881CC
:1011300099818617970769F48A819B81309719F006
:101140009383828304C09093390280933802FE0116
:1011500034C06817790738F44115510519F0841720
:10116000950708F4AC01FE018A819B819C01E9018D
:101170002097E9F641155105A9F1CA01861B970B85
:10118000049708F4BA01E0E0F0E02AC08D919C9148
:10119000119784179507F9F46417750781F412966F
:1011A0008D919C911397309719F09383828304C09B
:1011B0009093390280933802FD0132964FC0CA01E4
:1011C000861B970BFD01E80FF91F6193719302973E
:1011D0008D939C9343C0FD01828193819C01D90131
:1011E0001097A1F68091360290913702892B41F435
:1011F00080912702909128029093370280933602C3
:101200004091290250912A024115510541F44DB7F0
:101210005EB78091250290912602481B590B2091C0
:1012200036023091370224173507B0F4CA01821B09
:10123000930B8617970780F0AB014E5F5F4F8417C3
:10124000950750F0420F531F5093370240933602D8
:10125000F9016193719302C0E0E0F0E0CF01DF910A
:10126000CF910895CF93DF93009709F450C0EC011C
:1012700022971B821A82A0913802B09139021097EE
:1012800009F140E050E0AC17BD0708F1BB83AA8329
:10129000FE0121913191E20FF31FAE17BF0779F4E0
:1012A0008D919C911197280F391F2E5F3F4F3983E5
:1012B000288312968D919C9113979B838A83411565
:1012C000510571F4D0933902C093380220C01296B0
:1012D0008D919C911397AD01009711F0DC01D3CF54
:1012E000FA01D383C28321913191E20FF31FCE170C
:1012F000DF0769F488819981280F391F2E5F3F4FDE
:10130000FA01318320838A819B8193838283DF91D9
:10131000CF91089591119BC1803219F08950855069
:10132000D0F70895FC010590061621F00020D9F7AA
:10133000C00108953197CF0108950F931F93CF9364
:10134000DF938C01EB01009731F46115710519F4FD
:1013500020E030E038C081E090E06EE070E00E9474
:101360000B0BFC019C01009771F180E883832097AF
:1013700071F0D387C28781E8838380913A0290918C
:101380003B02892B21F4F0933B02E0933A020115D2
:101390001105C9F011870087838182608383809162
:1013A0003C0290913D02892B71F4F0933D02E09351
:1013B0003C0280913E0290913F02892B21F4F093F0
:1013C0003F02E0933E02C901DF91CF911F910F913F
:1013D0000895CF93DF93EC014B8140FF1AC046FF85
:1013E0000AC04F7B4B838E819F8101969F838E83A2
:1013F0008A81282F2BC042FF13C0E881F9818081A8
:10140000282F332727FD30952115310529F4406217
:101410004B832FEF3FEF1BC03196F983E88311C058
:10142000EA85FB85CE0119959C0197FF0AC09B8137
:101430002F5F3F4F11F080E201C080E1892B8B8349
:10144000E8CF8E819F8101969F838E8330E0C90112
:10145000DF91CF910895DF93CF93CDB7DEB79E0193
:10146000265F3F4F8E819F8168857985A9010E9403
:10147000E204CF91DF9108950F931F93CF93DF93F1
:101480008C01EB018B8181FF1BC082FF0DC02E817F
:101490003F818C819D812817390764F4E881F981A7
:1014A0000193F983E88306C0E885F985802F1995B3
:1014B000892B31F48E819F8101969F838E8302C098
:1014C0000FEF1FEFC801DF91CF911F910F9108958A
:1014D000EF92FF920F931F93CF93DF937C018B01C9
:1014E000DB0113968C9181FD03C0CFEFDFEF13C0BA
:1014F000C0E0D0E00BC0D8011896ED91FC9119978F
:10150000B8011995892B11F0CFEFDFEFF701819129
:101510007F01882381F7CE01DF91CF911F910F9139
:10152000FF90EF9008959C01FB01838180FF11C023
:1015300086FD0FC09FEF2F3F390759F0228380644B
:101540008F7D83838681978101979783868330E09F
:1015500002C02FEF3FEFC9010895FA01AA272830F2
:1015600051F1203181F1E8946F936E7F6E5F7F4F70
:101570008F4F9F4FAF4FB1E03ED0B4E03CD0670FEC
:10158000781F891F9A1FA11D680F791F8A1F911D3F
:10159000A11D6A0F711D811D911DA11D20D009F48F
:1015A00068943F912AE0269F11243019305D3193D1
:1015B000DEF6CF010895462F4770405D4193B3E0BA
:1015C0000FD0C9F7F6CF462F4F70405D4A3318F061
:1015D000495D31FD4052419302D0A9F7EACFB4E012
:1015E000A6959795879577956795BA95C9F70097CA
:1015F0006105710508959B01AC010A2E069457956B
:10160000479537952795BA95C9F7620F731F841FC1
:10161000951FA01D08950F931F93CF93DF93689F8D
:101620008001699F100D789F100D1124C8010E9440
:101630008508EC01009729F060E070E0A8010E94A5
:101640002A0BCE01DF91CF911F910F910895992719
:1016500088270895DC0101C06D9341505040E0F7A8
:061660000895F894FFCF8D
:1016660068656C6C6F20776F726C640A0D00476F4B
:1016760074206368617261637465723A2025632021
:0C16860025640A0D002000400200000056
:00000001FF
